:1000000000308A00DF280000831A0A28A500030EAA
:10001000A6000F288312A500030EA600A6140A0846
:10002000AD008A018313A50E0408A7002008A800CC
:100030002108A9002208AA002308AB002408AC006C
:1000400083128C308400001C27280C18D2288B1EA9
:100050002B280B194028270884002808A00029080D
:10006000A1002A08A2002B08A3002C08A4002D0838
:100070008A00260E83008312250EA6188316090017
:10008000B4140B118A112B282030DA00D601D701C5
:10009000D801D9015108A3005008A2004F08A100BF
:1000A0004E08A0000310201C63285208D6075308EE
:1000B0000318530FD70754080318540FD8075508CF
:1000C0000318550FD907D90CD80CD70CD60CA30C94
:1000D000A20CA10CA00CDA0B52280034A101A20141
:1000E000A001A3015408031D78285308031992287E
:1000F0001030D5000310D10DD20DA00DA30D540862
:100100002302031D852853082002031C8E28530850
:10011000A002031CA3035408A3020314A10DA20D03
:10012000D50B7A28000000343308D1003208D00003
:100130003108CF003008CE004130D500C630D400A1
:100140004E30D3006D30D200442039302007B0004B
:100150002108B100303003183130B1072208B20055
:10016000003003180130B2072308B3000030031831
:100170000130B3073208A0003308A100A201A30197
:100180003308D0003208CF003308D2003208D10043
:100190007F30D400FF30D3006E202008A100230858
:1001A000A2000034B70A370BDC28942022088F0005
:1001B00021088E003414B7010C108A112B288401F9
:1001C0001F308305713083168F0083121F1383162F
:1001D0001F109F101F119F11073083129900AF014C
:1001E0000130B000B101B201B3013410B410B70155
:1001F000F430B8000130B900BA00BB01F430BC00E3
:100200000130BD000A30BE00BF0140141F13831629
:100210001F149F101F119F111F169F161F1383126B
:100220009F171F1483160108C03903388100B530A9
:10023000831290000030A10004389200FF30831632
:1002400092000511831205110C30950007309900BA
:100250008316050806308312A000A00B2D2900008C
:1002600019088C11831699010C14C03083128B0469
:100270008B16713083168F008312341C9E293B0825
:10028000B9003A08B800AE018B1BAE178B1394204F
:10029000AE1B8B172208B6002108B500AE018B1BE0
:1002A000AE178B133608D2003508D1000330D400C6
:1002B000FF30D3006E20AE1B8B172008B50023083B
:1002C000B6003608BB003508BA00AE018B1BAE176E
:1002D0008B139420AE1B8B172208B6002108B500A3
:1002E000AE018B1BAE178B133608D2003508D10038
:1002F000D4010A30D3006E20AE1B8B172008B50046
:100300002308B600BF010A30BE003908BD00380816
:10031000BC00BB1F8E29B91F9A299029B91B9C29A3
:100320003B083902031C9C29031D9A2938083A020C
:1003300003189C2940149D2940103410B41CED2949
:10034000401CBE293E08BC023F08031C3F0FBD02F3
:10035000BD1FAD29BB1FB929AF29BB1BBD293D0856
:100360003B02031CBD29031DB9293C083A02031CAA
:10037000BD293B08BD003A08BC00D9293E08BC078E
:100380003F0803183F0FBD07BB1FC929BD1FD52953
:10039000CB29BD1BD9293B083D02031CD929031DCC
:1003A000D5293A083C02031CD9293B08BD003A086C
:1003B000BC003D08A2003C08A100A20CA10CA20CAC
:1003C000A10CA20C21089300A20C220C3039A00031
:1003D0001508CF3920049500B41083163C2963001A
:02400E00F43488
:00000001FF
